:100000000C94D9050C9411060C9411060C9411064D
:100010000C9411060C9411060C9411060C94110604
:100020000C9411060C9411060C9411060C94AF2A32
:100030000C945E2B0C9420250C9411060C94110644
:100040000C9411060C9411060C94D01D0C94A82548
:100050000C9411060C9411060C9411060C941106C4
:100060000C9411060C9411060C9411060C941106B4
:100070000C941106E709E709130A130A7B0A990A87
:10008000B10BB10BA40A3D0B4E0B4E0BDD1CDF1C5C
:10009000E41CE71CEA1CED1CF01CCB2BF22BEA2C19
:1000A000F22BEA2C3E2C612CEA2CB82CC72C290010
:1000B000C05CBE5CBF5C53005400550067005F002D
:1000C0006000610056005C005D005E005700590052
:1000D0005A005B0058006200620063005800010093
:1000E0000100010001000100010001000100010008
:1000F00001000100010001000100010001000100F8
:1001000001000100010001000100010001000100E7
:1001100001000100010001000100010001000100D7
:1001200001000100010001000100010001000100C7
:1001300001000100010001000100010001000100B7
:1001400001000100010001000100010001000100A7
:100150000100010001000100010001000100010097
:1001600001000100010001000100010001004445FF
:100170004255473A2064697361626C65642E0A00D7
:1001800044454255473A20656E61626C65642E0AAB
:10019000000A0025303258006C65645F7461736B2F
:1001A0003A20004F6E6573686F743A20616374691A
:1001B00076653A2025640A000A0025303862003A44
:1001C000200025303258000A722F6320303132333C
:1001D000343536370A00290A002575002F002575A9
:1001E000005D2800256400200025640020002564AF
:1001F0000020002564007C0025303258006D6F75AA
:1002000073656B6579205B62746E7C7820792076EB
:1002100020685D287265702F61636C293A205B004D
:100220006261636B6C69676874206272656174688F
:10023000696E672064697361626C650A006261635C
:100240006B6C6967687420627265617468696E6757
:1002500020656E61626C650A006261636B6C696740
:10026000687420627265617468696E6720746F6774
:10027000676C653A2025750A006261636B6C69677B
:10028000687420737465703A2025750A0062616392
:100290006B6C696768742064697361626C650A00DD
:1002A0006261636B6C6967687420656E61626C651E
:1002B0000A006261636B6C6967687420746F6767BA
:1002C0006C653A2025750A006261636B6C6967682A
:1002D000742064656372656173653A2025750A0050
:1002E0006261636B6C6967687420696E63726561D3
:1002F00073653A2025750A00000000000000000028
:1003000000000001010203040506080A0C0F111485
:10031000181C2024292E33393F464C535B626A71E6
:1003200079818A929AA2AAB2B9C1C8CFD5DCE1E795
:10033000EBF0F4F7FAFCFDFEFFFEFDFCFAF7F4F03B
:10034000EBE7E1DCD5CFC8C1B9B2AAA29A928A8103
:1003500079716A625B534C463F39332E2924201C45
:100360001814110F0C0A080605040302010100000D
:100370000000000000000000313A0964656C6179FA
:10038000282A31306D73293A2025750A323A0969D5
:100390006E74657276616C286D73293A2025750A32
:1003A000333A096D61785F73706565643A2025752D
:1003B0000A343A0974696D655F746F5F6D61783AEC
:1003C0002025750A353A09776865656C5F6D617837
:1003D0005F73706565643A2025750A363A09776857
:1003E00065656C5F74696D655F746F5F6D61783AA8
:1003F0002025750A00703A097072696E7420766162
:100400006C7565730A643A09736574206465666186
:10041000756C74730A75703A092B310A646E3A0967
:100420002D310A6C743A092B31300A72743A092D55
:1004300031300A4553432F713A09717569740A0ABC
:100440007370656564203D2064656C7461202A20AA
:100450006D61785F7370656564202A20287265700D
:10046000656174202F2074696D655F746F5F6D61C5
:1004700078290A77686572652064656C74613A2032
:10048000637572736F723D25642C20776865656CA7
:100490003D25640A53656520687474703A2F2F6592
:1004A0006E2E77696B6970656469612E6F72672F54
:1004B00077696B692F4D6F7573655F6B6579730A2B
:1004C000004D3E20004D25753A25733E20003F0A21
:1004D000003D2025750A003F0A0064656661756C61
:1004E00074730A0025750A003F0A000A092D205678
:1004F000616C756573202D0A00710A000A092D20B0
:100500004D6F7573656B6579202D0A003F00433E82
:1005100020004C25640A000A092D2053746174756B
:1005200073202D0A686F73745F6B6579626F6172F7
:10053000645F6C65647328293A20253032580A6B51
:100540006579626F6172645F70726F746F636F6CF4
:100550003A20253032580A6B6579626F6172645FA8
:1005600069646C653A20253032580A74696D657289
:100570005F72656164333228293A202530386C581F
:100580000A000A092D2056657273696F6E202D0AC4
:100590005649443A20307834453538284E6F7861D2
:1005A000727929205049443A203078303839392836
:1005B00032323029205645523A20307830303031AE
:1005C0000A4255494C443A20202846656220323878
:1005D0002032303232290A4F5054494F4E533A207C
:1005E0004C554641204D4F5553454B455920455894
:1005F0005452414B455920434F4E534F4C45204395
:100600004F4D4D414E4420343039360A4743433A2A
:1006100020352E342E30204156522D4C4942433A3B
:1006200020322E302E30204156525F415243483AFC
:100630002061767233350A000A092D20436F6E73EC
:100640006F6C65202D0A4553432F713A0971756906
:10065000740A6D3A096D6F7573656B65790A000AE6
:10066000092D204D61676963202D0A443A094465CC
:10067000627567204D65737361676520546F6767A6
:100680006C650A583A094D61747269782044656254
:100690007567204D6F646520546F67676C65202D0A
:1006A0002053686F77206B6579707265737365731B
:1006B00020696E206D617472697820677269640ABE
:1006C0004B3A094B6579626F6172642044656275CB
:1006D0006720546F67676C65202D2053686F772003
:1006E0006B65797072657373207265706F72740ACE
:1006F0004D3A094465627567204D6F7573652054E6
:100700006F67676C650A563A0956657273696F6E52
:100710000A533A095374617475730A433A09416381
:1007200074697661746520436F6E736F6C65204DDC
:100730006F64650A46312D4631303A095377697442
:10074000636820746F204C6179657220302D3920E8
:1007500028463130203D204C30290A302D393A09C5
:1007600053776974636820746F204C6179657220D7
:10077000302D390A47524156453A09537769746317
:100780006820746F204C6179657220302028616C7C
:100790007465726E617465290A423A094A756D7012
:1007A00020746F20426F6F746C6F616465720A45CC
:1007B00053433A094A756D7020746F20426F6F740D
:1007C0006C6F616465722028616C7465726E61740F
:1007D00065290A453A095072696E742045455052A0
:1007E0004F4D2053657474696E67730A42535041CC
:1007F00043453A09436C65617220454550524F4D5F
:100800000A006261636B6C696768745F636F6E6630
:1008100069672E7261773A20253032580A2E656E4C
:1008200061626C653A2025750A2E6C6576656C3AB6
:100830002025750A006B65796D61705F636F6E6668
:1008400069672E7261773A20253032580A2E737705
:1008500061705F636F6E74726F6C5F636170736CF5
:100860006F636B3A2025750A2E636170736C6F633A
:100870006B5F746F5F636F6E74726F6C3A20257577
:100880000A2E737761705F6C63746C5F6C67756957
:100890003A2025750A2E737761705F7263746C5FFE
:1008A000726775693A2025750A2E737761705F6CDF
:1008B000616C745F6C6775693A2025750A2E7377D1
:1008C00061705F72616C745F726775693A2025753B
:1008D0000A2E6E6F5F6775693A2025750A2E737749
:1008E00061705F67726176655F6573633A20257535
:1008F0000A2E737761705F6261636B736C617368FA
:100900005F6261636B73706163653A2025750A2EBF
:100910006E6B726F3A2025750A0064656275675FB9
:10092000636F6E6669672E7261773A2025303258A0
:100930000A2E656E61626C653A2025750A2E6D611E
:10094000747269783A2025750A2E6B6579626F6139
:1009500072643A2025750A2E6D6F7573653A2025ED
:10096000750A006565636F6E6669673A0A64656655
:1009700061756C745F6C617965723A2025750A0047
:100980003F000A6D6F7573653A206F66660A000A4C
:100990006D6F7573653A206F6E0A000A6B65796238
:1009A0006F6172643A206F66660A000A6B6579624D
:1009B0006F6172643A206F6E0A000A6D6174726929
:1009C000783A206F66660A000A6D61747269783A37
:1009D000206F6E0A000A64656275673A206F66666A
:1009E0000A000A64656275673A206F6E0A000A0A97
:1009F0004A756D70696E6720746F20626F6F746CDA
:100A00006F616465722E2E2E2000433E2000436CE1
:100A1000656172696E6720454550524F4D0A000A64
:100A2000002530325820006B6579626F6172645F17
:100A30007265706F72743A20005B735D005B575D86
:100A4000005B535D005B525D0008033200320030F2
:100A50000000000E034E006F007800610072007904
:100A60000000000403090409025B00030100A0FA6E
:100A70000904000001030101000921110100012204
:100A8000400007058103080001090401000103007B
:100A90000000092111010001227B000705820320CB
:100AA00000010904020002030000000921110100F5
:100AB000012222000705830320000107050303200C
:100AC00000011201000200000008584E99080100C0
:100AD000010200010631FF0974A101097515002604
:100AE000FF009520750881020976150026FF009504
:100AF0002075089102C005010902A10185020901C2
:100B0000A10005091901290815002501950875019D
:100B100081020501093009311581257F950275088B
:100B2000810609381581257F950175088106050C18
:100B30000A38021581257F950175088106C0C00518
:100B4000010980A101850319012AB700150126B703
:100B500000950175108100C0050C0901A1018504F3
:100B600019012AA002150126A00295017510810025
:100B7000C005010906A101050719E029E7150025AF
:100B80000195087501810295017508810105071914
:100B90000029FF150026FF0095067508810005084D
:100BA00019012905950575019102950175039101BA
:100BB000C00011241FBECFEFD4E0DEBFCDBF04B60E
:100BC00003FE18C08091BF029091C002A091C102A3
:100BD000B091C2028730904BA740B04B59F41092AD
:100BE000BF021092C0021092C1021092C202E0E055
:100BF000F8E3099511E0A0E0B1E0EAEFFBE502C0FF
:100C000005900D92A43FB107D9F722E0A4EFB1E01F
:100C100001C01D92AF3BB207E1F70E94EC170C94A4
:100C2000FB2D0C940000FF93EF93E091F401F09101
:100C3000F501309709F00995EF91FF910895FC01B6
:100C40008591803011F0EFDFFBCF0895FF27E0E2C0
:100C500030E247FF0CC0419597FF09C0EDE2609577
:100C6000709580959095611D711D811D911D27FFC7
:100C700002C0219530E350E2AA27660F771F881F34
:100C8000991FAA1FA41710F0A41B63955A95A9F7E2
:100C9000AA3008F0A95FA05DAF93F39561157105C7
:100CA0008105910541F7ED3211F4EF93F395F217B9
:100CB00018F43F93F395FBCF8F91B5DFFA95E1F7E9
:100CC0000895E991F9918591803021F0853219F0EC
:100CD000AADFF9CF089520E0E89455915532C1F389
:100CE000503311F4689455915A3348F4505390F3AB
:100CF000220F022E220F220F200D250FF4CF0EF40B
:100D0000219589919991533619F3533729F1533528
:100D100059F1BC0188279927E8945C3621F4899120
:100D2000999168945591543639F446EF7EF077FFE7
:100D30000DC08FEF9FEF0AC055374AE039F05835A4
:100D400040E121F0523642E009F00895FF93EF931D
:100D50007DDFEF91FF91B7CFFF93EF93FC0181917E
:100D60008030B9F360DFFBCFFF93EF9368DFF1CF03
:100D7000DF93CF93CDB7DEB72596A3DFCF91DF9179
:100D800008953E9A0C94AF16CF93C82F0E94D207B5
:100D9000882329F0C0FF02C0469A01C0469881E02E
:100DA000CF91089581E0089581E008950C94D406D0
:100DB00008950C94D8061F93CF93DF9300D000D0F2
:100DC0001F92CDB7DEB749835A836B833091F70109
:100DD00089819A81311114C0662359F0222349F088
:100DE0000E94F10D182F682F89819A810E94970D1A
:100DF00003C00E94C50D182F69817A81812F04C01C
:100E00000E94F10D69817A810F900F900F900F90E1
:100E10000F90DF91CF911F910C942815FC01262F84
:100E2000408151816281738184810C94DB0681E071
:100E30000895CF93DF93EC0160E00E940E07BE019E
:100E4000DF91CF910C94D9060C94C1060C94AD1689
:100E500008950E94410C0E9428072FEF84E39CE034
:100E6000215080409040E1F700C000000C94CE2556
:100E70000F931F93CF93DF938C0161E00E940E07C5
:100E8000EC01B8010E94D606882309F462C0B801BB
:100E9000CE010E94CE1C882309F45BC0B801CE01AC
:100EA0000E94AE23882309F454C0B801CE010E94E9
:100EB000741E882309F44DC0B801CE010E940A2394
:100EC000882309F446C0F80182818823D9F1CF3DF7
:100ED0008CE5D80779F140F4C115FCE5DF0791F006
:100EE000C130DC4591F02EC0CC35EDE5DE0741F197
:100EF000CD35FDE5DF0709F1CB35DD4519F50E945C
:100F0000841220C00E94290724C080916902C82F42
:100F1000C095C170C0FB80F980936902CC2329F091
:100F200080E891E00E941F0614C08EE691E00E94C6
:100F30001F0610C00E9438130CC00E947B1202C012
:100F40000E948712C801DF91CF911F910F910C94DD
:100F5000D206C0E08C2FDF91CF911F910F910895A1
:100F60000E94032580E00E94841D0C94DE070E94ED
:100F7000861B0E94E1070C9409258295982F937394
:100F8000292F220F220F982F9C7C96959695922BB5
:100F9000892F8575880F9A7A9695892B08950895DB
:100FA0000C94CF0781E008950895CF93C82F0E9435
:100FB000D0078C2F0E94C406CF91089580E00C9436
:100FC000D5070E940A240C94D507CF930E940A24C7
:100FD000C82F8091F601C81741F1C093F6018091A6
:100FE000690282FF1EC080FF04C088E991E00E9470
:100FF0001F068091690280FF0CC01F92CF9383E986
:1010000091E09F938F930E94B8060F900F900F90DE
:101010000F908091690280FF04C081E991E00E94F5
:101020001F068C2FCF910C94D507CF910895CF93A5
:10103000DF93CDB7DEB72B970FB6F894DEBF0FBEA8
:10104000CDBF4F83588769877A878B8761110E944C
:10105000B3119E012F5F3F4F86E0F90111928A95EF
:10106000E9F785E0FE013796D90101900D928A9546
:10107000E1F789819A814C815D81452B31F09F3F59
:1010800031F491E08F3F19F403C091E001C090E08A
:1010900090FF09C049815A816B817C818D819E813D
:1010A0000E94CF1005C0C9010E9417078111F2CF1D
:1010B0002B960FB6F894DEBF0FBECDBFDF91CF9158
:1010C0000895FC01808191810E94330E0895CF9391
:1010D000882309F4A9C0C82F8238C1F40E940A24C9
:1010E00081FDA2C069E380910201909103010E94F9
:1010F000DB240E94D5112FEF81EE94E02150804037
:101100009040E1F700C0000069E319C0833801F5A1
:101110000E940A2480FD88C063E5809102019091BD
:1011200003010E94DB240E94D5112FEF81EE94E091
:10113000215080409040E1F700C0000063E58091BD
:101140000201909103010E94DD24CF910C94D511EE
:101150008438C1F40E940A2482FD66C067E480914D
:101160000201909103010E94DB240E94D5112FEF10
:1011700081EE94E0215080409040E1F700C00000F3
:1011800067E4DDCF8CEF8C0F813AF8F48C2F0E944E
:10119000B322811149C06C2F80910201909103010B
:1011A0000E94A524882349F06C2F80910201909120
:1011B00003010E94DD240E94D5116C2F8091020151
:1011C000909103010E94DB24C0CF80E28C0F883015
:1011D00048F4C77081E001C0880FCA95EAF70E9401
:1011E0009611B3CFEBE5EC0FE33040F4F0E0E75BB2
:1011F000FE4F808190E0CF910C946D24E8E5EC0FD8
:10120000E73150F4F0E0EE0FFF1FE55EFE4F808106
:101210009181CF910C948324CD3E30F08C2F0E948D
:101220007918CF910C944B19CF910895882309F424
:1012300064C0823879F40E940A2481FF5EC069E3A9
:1012400080910201909103010E94DB240E94D5113C
:1012500069E310C08338B1F40E940A2480FF4DC0B6
:1012600063E580910201909103010E94DB240E94BA
:10127000D51163E580910201909103010E94DD2464
:101280000C94D511843879F40E940A2482FF35C069
:1012900067E480910201909103010E94DB240E9487
:1012A000D51167E4E7CF9CEF980F913A10F4682FBF
:1012B000E1CF90E2980F983050F4877091E001C030
:1012C000990F8A95EAF7892F0E949C11D9CF9BE547
:1012D000980F933020F480E090E00C946D2498E512
:1012E000980F973120F480E090E00C9483248D3E99
:1012F00020F00E94D4180C944B1908951F93CF939B
:10130000DF93182FEB010E946708209741F08FE9C7
:101310009FE00197F1F700C000002197F6CF812FE1
:10132000DF91CF911F910C941609893319F060E079
:1013300070E002C060E570E00C947E09882321F023
:101340000E9496110C94D5110895882321F00E94D3
:101350009C110C94D5110895CF92DF92EF92FF92D9
:101360000F931F93CF93DF937C01D62FC72FFC01E0
:101370001281058102950F700E948C118823B9F0AB
:101380001123A9F08C2F807F803421F080E28D0F13
:10139000883068F08091A00282FD09C082E00E943E
:1013A00035120E948C1191E0D82ED92601C0D12C83
:1013B000CC2EC2948FE0C8228C2D90E08C30910509
:1013C00008F0CFC1FC01E65CFF4F0C94A62D8C2FDA
:1013D000807FCF70882311F0C295C07F112399F0D0
:1013E000CC2309F4AAC180E28D0F883010F0D1110E
:1013F00004C08C2F0E94961103C08C2F0E94A6114E
:101400000E94D5119AC18D2F0E941609CC2309F490
:10141000A8C180E28D0F883038F1DD2329F18C2FAF
:101420000E94AC1124C08C2F807FCF70803211F0CD
:10143000C295C07FDD2319F0D130A1F13DC080916C
:10144000A00282FF17C0112349F0CC2329F08C2F72
:101450000E9496110E94D51180E070C180E00E9428
:101460001609CC2309F47DC18C2F0E949C110E9487
:10147000D51177C1112371F0002341F0013031F40F
:101480000E94B6118C2B0E94BE116BC10E94B61136
:101490008C2B1DC0002319F0013009F462C10E9499
:1014A000CB1125C0112321F0063008F05AC10EC01F
:1014B000053008F056C11BC0112361F0002331F044
:1014C000F701858180FF39C18F7085838C2F0E9441
:1014D0009E0947C1002359F0D93309F03FC1FFEFFE
:1014E00007EE13E0F15000401040E1F735C18C2FBA
:1014F0000E94A50936C18C2F86958695837019F0B8
:10150000813061F02EC1112321F08D2F9C2F93701B
:1015100002C080E090E00E946D242BC1112321F0D5
:101520008D2F9C2F937002C080E090E00E94832456
:1015300020C18D2F112319F00E94791802C00E943A
:10154000D4180E944B1915C18C2F837009F047C025
:1015500011110BC12D2F229526952770220F220FD6
:101560006D2F6F70862F90E0A0E0B0E0022E04C0D7
:10157000880F991FAA1FBB1F0A94D2F7D4FF10C06F
:101580004FE050E060E070E004C0440F551F661F5C
:10159000771F2A95D2F7409550956095709503C0B6
:1015A00040E050E0BA01C695C695C3708A019B0120
:1015B000082B192B2A2B3B2BC901B801C23049F04B
:1015C00058F4C13019F00E94AD0CCFC00E949B0CA2
:1015D000CCC00E94BF0CC9C00E94990CC6C0112388
:1015E00019F08C2F817001C08695882309F4BDC045
:1015F0002D2F229526952770220F220F6D2F6F70A9
:10160000862F90E0A0E0B0E0022E04C0880F991F62
:10161000AA1FBB1F0A94D2F7D4FF10C04FE050E0BE
:1016200060E070E004C0440F551F661F771F2A95C5
:10163000D2F7409550956095709503C040E050E01A
:10164000BA01C695C695C3708A019B01082B192B58
:101650002A2B3B2BC901B801C23049F058F4C130E4
:1016600019F00E94720D81C00E94600D7EC00E9420
:10167000840D7BC00E94D30C78C0CF70112339F049
:101680008C2F0E94F90C8D2F0E949E096EC08D2F09
:101690000E94A5098C2F0E941A0D67C0D23F21F12C
:1016A00028F4D03F41F0D13FC1F043C0D33F19F1FE
:1016B000D43F79F03EC0112341F0053008F051C00D
:1016C0008C2F8F710E943F0D4CC0063008F049C02E
:1016D000F7CF8091A00282FF18C0112339F08C2F20
:1016E0008F710E94F90C3DC01123C9F38C2F8F71AB
:1016F0000E941A0D36C0112329F08C2F8F710E9481
:10170000E40C2FC00E94DF0C2CC0112349F0CF71D4
:101710008C2F0E94F90C63E08C2F0E941A1221C0BA
:1017200081E00E9435120230E0F082E00E94351222
:1017300018C0112331F0002391F28D2F0E94670809
:1017400010C0002399F2D93349F41FEF27EE33E09C
:10175000115020403040E1F700C000008D2F0E9462
:10176000160988EF8C0D843020F40E940A240E9410
:10177000D507DD20C9F00E94881180FD15C0F70152
:1017800012820E9482110E94F90CC7010E94F50B7F
:101790000E948211DF91CF911F910F91FF90EF90E6
:1017A000DF90CF900C941A0DDF91CF911F910F9184
:1017B000FF90EF90DF90CF9008950F931F93CF93FA
:1017C000DF93EC01688179818A810E943E0E8C0151
:1017D0000E94960D0E94870CB801CE010E94AC09B0
:1017E000DF91CF911F910F910895CF93DF93EC017B
:1017F000988189812B813C81232B31F08F3F31F4FB
:1018000081E09F3F19F403C081E001C080E080FDCA
:101810001DC0CE010E943807811110C00E948C119A
:101820008823A1F08A81882389F08091A00282FD1B
:101830000DC082E0DF91CF910C943512CE010E9451
:10184000DD0BCE01DF91CF910C941907DF91CF9181
:10185000089580E090E00E946D2480E090E00E9476
:1018600083240E94B3110E94D5110E940C1B0C947A
:101870004B1980910201909103010E94DF240C9486
:10188000290C0E94A3110C94390C92959F709630EC
:1018900079F010F4925001C09A50923068F4803F71
:1018A00069F018F4883E40F409C0843F29F406C06A
:1018B000883E20F0813F11F080E0089581E0089596
:1018C000FC01808191810E94330E0E94450C089595
:1018D000CF93DF9300D000D01F92CDB7DEB70F902B
:1018E0000F900F900F900F90DF91CF910895CF93AD
:1018F000DF9300D000D000D0CDB7DEB726960FB66C
:10190000F894DEBF0FBECDBFDF91CF91089508954B
:1019100008950C94880C0C94890C0E948B0C609395
:101920000B0270930C0280930D0290930E020C94A4
:10193000290C0C948D0C0F931F9300910B021091A6
:101940000C0220910D0230910E02602B712B822B24
:10195000932B1F910F910C948D0C0F931F9300915B
:101960000B0210910C0220910D0230910E026023A7
:101970007123822393231F910F910C948D0C0F934D
:101980001F9300910B0210910C0220910D023091D7
:101990000E0260277127822793271F910F910C94C5
:1019A0008D0C0C94880C0E94D10C609307027093EC
:1019B00008028093090290930A020C94290C60E0BB
:1019C00070E0CB010C94D30C0F931F9341E050E0D7
:1019D00060E070E08A019B0104C0000F111F221F0C
:1019E000331F8A95D2F7C901B8011F910F910C944A
:1019F000D30C0F931F9341E050E060E070E004C00F
:101A0000440F551F661F771F8A95D2F780910702F2
:101A100090910802A0910902B0910A028A019B01EB
:101A2000082B192B2A2B3B2BC901B8011F910F91B1
:101A30000C94D30C0F931F9341E050E060E070E0F2
:101A400004C0440F551F661F771F8A95D2F7409533
:101A50005095609570958091070290910802A09131
:101A60000902B0910A028A019B01082319232A2343
:101A70003B23C901B8011F910F910C94D30C0F9314
:101A80001F9341E050E060E070E004C0440F551F38
:101A9000661F771F8A95D2F78091070290910802FE
:101AA000A0910902B0910A028A019B010827192717
:101AB0002A273B27C901B8011F910F910C94D30C21
:101AC0000F931F93009107021091080220910902C1
:101AD00030910A02602B712B822B932B1F910F9157
:101AE0000C94D30C0F931F930091070210910802DE
:101AF0002091090230910A026023712382239323EB
:101B00001F910F910C94D30C0F931F930091070218
:101B1000109108022091090230910A026027712772
:101B2000822793271F910F910C94D30C0895262F91
:101B3000990F990F890F982F9770A1E001C0AA0FF4
:101B40009A95EAF786958695869590E065E070E02F
:101B50000E94262DFC01E850FE4F40E050E0622F2D
:101B600070E090819B01042E02C0369527950A945F
:101B7000E2F72170219529272A23292721934F5FF6
:101B80005F4F4530510569F70895990F990F890FF7
:101B9000A82FA77086958695869590E065E070E001
:101BA0000E94262DBC0140E050E080E0FB01E40FE4
:101BB000F51FE850FE4F208130E00A2E02C0369516
:101BC00027950A94E2F721703327042E01C0220FD3
:101BD0000A94EAF7822B4F5F5F4F4530510531F78A
:101BE0000895BF92CF92DF92EF92FF920F931F93CF
:101BF000CF93DF938C01C0900702D0900802E09051
:101C00000902F0900A0280910B0290910C02A091BF
:101C10000D02B0910E02C82AD92AEA2AFB2ACFE186
:101C2000D0E0D701C6010C2E04C0B695A7959795B4
:101C300087950A94D2F780FD04C0219790F7B12CC4
:101C400007C0BC2EB8018C2F0E943E150197A9F346
:101C50008B2DDF91CF911F910F91FF90EF90DF902F
:101C6000CF90BF900895CF93DF93EC010E94F10DC8
:101C7000BE010E943E15DF91CF9108951F93CF932F
:101C8000DF93EB019091F701992321F0CB010E94A2
:101C9000330E13C0882349F0CB010E94F10D182F99
:101CA000682FCE010E94970D04C0CB010E94C50D84
:101CB000182FBE01812F0E943E15DF91CF911F91F9
:101CC0000895CF93DF93C0910F0280911002C8173F
:101CD000A1F0D0E0CE0166E070E00E94262DFC016C
:101CE000EF5EFD4F408151816281738184819581D6
:101CF0000E94770C2196C770E8CFDF91CF910895AD
:101D0000409141025091420260914302709144021D
:101D100080914502909146020C94770CFF920F93AC
:101D20001F93CF93DF938091460282958F7009F0C5
:101D300062C080914302882309F45DC020910F02A4
:101D4000F09010021091410200914202A0914402D1
:101D5000B091450281E01F3F09F080E0C091000191
:101D6000D0910101482F2F1509F445C0109721F09B
:101D70000F3F21F080E003C081E001C0842F30E0FC
:101D800080FD35C0C90166E070E00E94262DFC018F
:101D9000EF5EFD4F818180132AC08081811327C0AF
:101DA0008281811124C0838194818A1B9B0B8C17B3
:101DB0009D07E8F4809146028F708061809346020F
:101DC000C90166E070E00E94262DFC01EA5EFD4F2D
:101DD00090819F709061908381E492E00E94F50B66
:101DE000DF91CF911F910F91FF900C94610E2F5FA7
:101DF0003F4F2770B8CFDF91CF911F910F91FF9088
:101E000008959F92AF92BF92CF92DF92EF92FF928E
:101E10000F931F93CF93DF93CDB7DEB761970FB6C4
:101E2000F894DEBF0FBECDBF8C0185E0F801DE0166
:101E30001D9601900D928A95E1F7F801E28090914C
:101E40004102309142026091440270914502611555
:101E5000710531F03F3F31F481E09F3F19F403C039
:101E600081E001C080E0F82FF1709F2E80FD47C116
:101E7000F80140812181A380B48081E4C82E82E0F2
:101E8000D82EF0904302F501E61BF70B609100019C
:101E900070910101FF2009F4DCC080914602582FA7
:101EA000507FE617F70708F096C0511155C023136D
:101EB00013C0491311C0FE2CE1100EC08F70806159
:101EC000809346020E94800EC6010E94F50B80910D
:101ED0004602F801858350C1AB2831F02F3F31F421
:101EE00081E04F3F19F403C081E001C080E080FD34
:101EF00003C081E08E2502C080E090E0F82FF170F1
:101F0000FF2E80FF1FC0E0910F0230911002E317F7
:101F100009F410C1F0E0CF0166E070E00E94262DC8
:101F2000DC01AF5EBD4F11968C911197281307C04D
:101F30008C91481304C012968C91E81203C031961C
:101F4000E770E5CFFE2CEE2009F416C18091460221
:101F500081608093460254C0231306C0491304C015
:101F6000E11002C0F80199C0C8010E94600C8823EA
:101F700061F1EE2051F120914602822F82958F70FF
:101F800090E0029774F0809141029091420298870C
:101F90008F831986BB86AA862C87CE0107960E945E
:101FA000F50B86E0F801A1E4B2E001900D928A956C
:101FB000E1F70E948E0E0E94800E0AC0231711F1D5
:101FC000C8010E94600C81112CC0C8010E94F50B51
:101FD000FF24F394D1C05111F1CF7A2DB98AA88A88
:101FE000522F6E2D89890E94680C81E492E00E9434
:101FF000F50B86E0F60111928A95E9F70E94800EB2
:10200000F12CBAC04913DCCFE110DACFF801858397
:10201000C8010E94F50B86E0F60111928A95E9F756
:10202000ABC0EE2091F220914602822F82958F70F4
:1020300090E002970CF4B5CF80914102909142025A
:102040009A8389831B82BD82AC822E83CE01019646
:10205000A6CFE617F70708F044C0FE2CEE2009F4DF
:10206000B4CF231330C049132EC02091460220FD67
:1020700021C0822F82958F70482F50E04115510565
:10208000C9F0F80125834F30510541F08F5F982F3B
:102090009295907F822F8F70892B8583C8010E9433
:1020A000F50B86E0F801A1E4B2E001900D928A956B
:1020B000E1F73DC086E0F801A1E4B2E001900D92A5
:1020C0008A95E1F759C0C8010E94600C811169CF5F
:1020D00080914602816080934602C8010E94F50B00
:1020E0004BC07A2DB98AA88A522F6E2D89890E94F9
:1020F000680C86E0F60111928A95E9F718C0EE2087
:1021000009F463CFC8010E94600CF82E882309F4FB
:102110005CCF86E0F801A1E4B2E001900D928A95CF
:10212000E1F781E492E00E9461080E948E0E0E9415
:10213000800E22C04D872E878D859E850E94330E8E
:10214000292F22952F70223028F49F7039F08111A9
:1021500005C00BC0243028F49F7049F4805E88309D
:1021600020F0C8010E94F50B9F2CF92C05C0F80146
:102170009581907F99F7F9CF8F2D61960FB6F894DE
:10218000DEBF0FBECDBFDF91CF911F910F91FF90AA
:10219000EF90DF90CF90BF90AF909F900895CF9336
:1021A000DF93CDB7DEB72C970FB6F894DEBF0FBE26
:1021B000CDBF4F83588769877A878B879C87CE01ED
:1021C00007960E94010F8823D1F09F8188852A8578
:1021D0003B85232B31F08F3F31F481E09F3F19F491
:1021E00003C081E001C080E080FD6FC04F81588551
:1021F00069857A858B859C850E94770C66C086E010
:10220000FE013796DE01119601900D928A95E1F755
:10221000FF81E8856A857B856115710531F0EF3FA7
:1022200031F481E0FF3F19F403C081E001C080E098
:1022300080FD4BC08091100290E09C012F5F3F4FCA
:102240002770332740910F0250E02417350709F417
:1022500043C0F983EA837D836C8366E070E00E946B
:10226000262DDC01AF5EBD4F96E0FE013196019058
:102270000D929A95E1F7209310020E94610E25C0FD
:1022800090E066E070E00E94262D8F5E9D4F0E94D8
:10229000010F882371F180910F0290E066E070E0F9
:1022A0000E94262DFC01EF5EFD4F4081518162812D
:1022B0007381848195810E94770C80910F0290E058
:1022C00001968770992780930F0280910F02909159
:1022D00010028913D5CF0DC00E94410C109210023C
:1022E00010920F02E1E4F2E086E0DF011D928A9590
:1022F000E9F72C960FB6F894DEBF0FBECDBFDF9185
:10230000CF91089580914F02859585958595089583
:1023100080914F028770089590914F02977081E0ED
:1023200009F480E0089580915A02089590915A022C
:10233000892B80935A020895809590915A0289239F
:1023400080935A02089510925A020895909159026A
:10235000892B809359020895809590915902892381
:102360008093590208951092590208958091500265
:10237000089508950C94B9110C94BA119091A0028B
:1023800092FD08C090915002981721F0809350025E
:102390000C94BC11089580915002882329F010926A
:1023A000500280E00C94BC110895CF93DF93E0912C
:1023B0000201F091030180915A028083E0910201B1
:1023C000F0910301908180915902892B8083809143
:1023D0005002882381F0E0910201F0910301908185
:1023E000892B808380910201909103010E9499249E
:1023F00081110E94CB11C0910201D091030148E0EC
:1024000050E067E472E0CE010E94AC2D892B69F0A8
:1024100088E0FE01A7E4B2E001900D928A95E1F711
:10242000CE01DF91CF910C941624DF91CF910895C6
:102430000C94B9119091A00292FD10C0982F990FA1
:10244000990F990F692B60934F020E94F90C8091AC
:102450004F028595859585950C9418120C94F90C6E
:1024600010924F0280E00C94181220914F02809538
:10247000822380934F02982F977099F430E0482F71
:10248000082E000C550B2417350759F09091A00227
:1024900092FD07C08595859585950E941A0D0C942F
:1024A00030120895CF939091A00292FB222720F939
:1024B0002817F9F0C82F892FC0FB82F98093A0025A
:1024C00080919F029091A0020E94B41282E00E942B
:1024D00035128091690280FF0CC01F92CF9383EA6E
:1024E00091E09F938F930E94B8060F900F900F90EA
:1024F0000F90CF9108958091A00282FB882780F9E8
:1025000091E089270C94521281E00C94521280E0E1
:102510000C9452126FEF7FEF80E090E00C94E52D69
:1025200080E090E00E94C12D21E0893E9E4F09F09D
:1025300020E0822F089582E090E00C94B92D83E092
:1025400090E00C94B92DCF9384E090E00E94B92DD7
:10255000C82F82E290E00E94B92D2C2F30E0A90113
:10256000582BCA01CF910895CF93C92F682F84E0CB
:1025700090E00E94C72D6C2F82E290E0CF910C94E6
:10258000C72DAB01BC018FE090E00C94D92DAB01BD
:10259000BC0183E190E00C94D92D60E070E0CB01A8
:1025A0000C94C71260E070E0CB010E94C1120C9441
:1025B000CD1269EE7EEF80E090E00E94E52D60E0B4
:1025C00082E090E00E94C72D60E083E090E00E94EE
:1025D000C72D10920B0210920C0210920D02109255
:1025E0000E0260E084E090E00E94C72D60E082E28D
:1025F00090E00E94C72D60E085E090E00E94C72D2A
:1026000060E086E090E00E94C72D6FEF87E090E0E9
:102610000E94C72D40E050E0BA0188E090E00E949F
:10262000D92D60E08DE090E00E94C72D40E050E0A1
:10263000BA0188E190E00E94D92D60E087E190E046
:102640000E94C72D40E050E0BA018CE190E00E946A
:10265000D92D60E070E080E290E00E94E52D40E03E
:1026600050E0BA0188E190E00E94D92D0C94D2127A
:102670000C94D912682F8EE090E00C94C72D0E9424
:102680008D25609365027093660280936702909334
:102690006802609361027093620280936302909378
:1026A0006402089581E008950C94521308950C94E7
:1026B00056130C9456130C9459130C9456130C94F3
:1026C0005D130C94561388EA97E20E9400240E943E
:1026D00061130C945F130E9457130C9456130E94BD
:1026E00032160E94D4070C945E1E0E9478250E9428
:1026F0004C170E946F130E94861B0C945B138F92E1
:102700009F92AF92BF92CF92DF92EF92FF920F9380
:102710001F93CF93DF93CDB7DEB72A970FB6F89408
:10272000DEBF0FBECDBF0E946117982E81110E949F
:102730003F138BE5A82E82E0B82E00E010E0802E3B
:10274000802F0E945616D82EF501C1905F01C82631
:10275000B1F40F5F1F4F0630110589F78FEF8983A2
:102760008A831B820E9481258160782F9D838C83C0
:1027700049815A816B818D810E9417082FC08091F9
:10278000690281FD0E945C16E12CFF24F3948C2DDC
:102790008F21F1F00E945413882399F0EE828F82EA
:1027A000DF2081E009F480E088870E948125816034
:1027B000782F9A8789874E815F8168858A850E94F4
:1027C0001708F801E55AFD4F8081F826F08206C00F
:1027D000E394FF0CF4E0EF12DACFBBCF81E091106D
:1027E00001C080E02A960FB6F894DEBF0FBECDBFC1
:1027F000DF91CF911F910F91FF90EF90DF90CF90DD
:10280000BF90AF909F908F9008950E947F130E9479
:10281000BA1D0E94EB190C94E507CF93DF930E9439
:102820004315EC01811521E5920708F045C081159B
:1028300030E5930708F094C0883E910528F5803E66
:10284000910508F001C1883A910570F4853A910527
:1028500008F07CC08130910509F475C008F4F1C01E
:10286000049708F0F1C0EDC08F3B910508F0E9C076
:10287000C85AD0E0CC0FDD1FC45BDE4F0990D88171
:10288000C02DCE019464E1C0811540E2940758F454
:10289000811551E0950708F0D7C08D3E910508F4E9
:1028A000D0C09065D2C0C11580E4D80708F4C9C073
:1028B000DF70CE01906AC9C0811525E59207A8F4A2
:1028C000811534E5930708F09EC0811543E5940710
:1028D00008F081C0811552E5950708F064C0D82F33
:1028E000CC27CE01816F906AB0C0C11589E5D807A9
:1028F000A0F4C11528E5D20708F08BC0C11536E554
:10290000D30708F09EC08C2F0E94D7158F7190E0DE
:10291000D82FCC27CE01906298C0C1154AE5D407C4
:1029200008F47DC0CE0190568115904208F089C010
:102930008D2F8F710E94D715DD27D0628F71AE0168
:10294000582BCA0182C081E090E07FC0C55AD0E018
:10295000C658DE4F8881C82FD0E0CE01906475C084
:10296000F4E096958795FA95E1F7282F23703C2F90
:10297000337081E090E002C0880F991F3A95E2F72A
:102980009C68AC01522B9C2F9F7096959695892F31
:1029900090E0EC01A5E0CC0FDD1FAA95E1F7CA019C
:1029A0008C2B9D2B52C08370992721E030E002C010
:1029B000220F331F8A95E2F79C2F96959695C92F83
:1029C000D0E075E0CC0FDD1F7A95E1F7C22BD32B59
:1029D000CE019C683AC08370992721E030E002C0A4
:1029E000220F331F8A95E2F79C2F96959695C92F53
:1029F000D0E065E0CC0FDD1F6A95E1F7C22BD32B49
:102A0000CE019A6822C0D82FCC27CE01846F906A5D
:102A10001CC0DC2FCC27CE01806F906A16C08C2F93
:102A20008F700E94D71594E0D695C7959A95E1F7D7
:102A3000CF70D0E0DC2FCC27D0699E01282BC901B4
:102A400004C080E090E001C0CE01DF91CF910895F5
:102A50009B0190E066E070E00E94262D830F911D9F
:102A6000FC01EE0FFF1FEE0FFF1FE20FF11DEE0F37
:102A7000FF1FE255FF4F8591949108950E942815FC
:102A80000E940D1408958238910569F1B0F48133E4
:102A9000910509F46DC048F48932910509F463C0C9
:102AA0008A32910509F469C008958533910509F4C6
:102AB00055C089339105B9F00895833E910569F1B8
:102AC00038F4803E9105B1F0823E910509F10895F8
:102AD000863E9105A9F1873E9105B9F1843E9105A5
:102AE00009F064C023C020919F0220FD4FC021FD4A
:102AF0004DC0089580919F0280FD44C08091A00246
:102B000080FF44C080919F0284FD42C083EE4DC08F
:102B100080919F0282FF38C0F5CF80919F0282FD95
:102B200033C08091A00280FD31C0ECCF8091A00223
:102B300081FF32C080919F0284FD2AC087EE35C09C
:102B400080919F0283FF26C0F5CF80919F0283FD75
:102B500021C08091A00281FD1FC0ECCF80919F0217
:102B600085FD1CC01DC080919F0285FD19C016C047
:102B700080919F0286FD16C017C080919F0286FD3E
:102B800013C010C089E311C082EE0FC080EE0DC0EB
:102B900080E00BC086EE09C084EE07C089E205C064
:102BA00085E303C08AE201C081E390E0089590913B
:102BB0009F0292FF0DC0282F2871283019F4877FBB
:102BC000846006C0282F2471243011F48B7F886024
:102BD00093FF0DC0282F2871283119F4877E846156
:102BE00006C0282F2471243111F48B7E8861209136
:102BF000A00220FF0DC0382F3871383019F4877FBC
:102C0000816006C0382F3171313011F48E7F8860B9
:102C100021FF0DC0282F2871283119F4877E81618A
:102C200006C0282F2171213111F48E7E886194FD18
:102C3000877E08950C948A120E9461178FE39CE9A5
:102C40000197F1F700C000000E94611780E00E9428
:102C5000561680FF04C00E941A160C94CE250895C3
:102C60000C941C160E949012811102C00E9438130D
:102C70000E949B12809369020E94A3129093A0026B
:102C800080939F020E9430160E949F12682F70E06E
:102C900080E090E00E94990C609107027091080218
:102CA0008091090290910A020C94D10CE82FF0E077
:102CB000E955FD4F80810895CF92DF92EF92FF9208
:102CC0000F931F93CF93DF9387EC91E00E941F0631
:102CD00087EAE82E82E0F82EC0E0D0E092ECC92E20
:102CE00091E0D92E0AEB11E0DF93CF93DF92CF92E0
:102CF0000E94B8068FEB91E00E941F06F7018191B8
:102D00007F010E94BD071F928F931F930F930E9414
:102D1000B80688EB91E00E941F0621968DB79EB7FA
:102D200008960FB6F8949EBF0FBE8DBFC630D10572
:102D3000D9F6DF91CF911F910F91FF90EF90DF9027
:102D4000CF90089580EA8A95F1F7089500C008951C
:102D50000C94A21608950C94AA160C94AB160C941D
:102D6000AA16F894E82FE295EF70F0E031A1282F31
:102D70002F7081E090E001C0880F2A95EAF7982F24
:102D80009095932391A392A1892B82A3789408957F
:102D90000F931F93CF93DF93C1E8D1E089918F3FC9
:102DA00011F00E94B11681E0C738D807B9F7CDE716
:102DB000D1E001E811E089918F3F11F00E94B11636
:102DC0000C171D07C1F7DF91CF911F910F91089547
:102DD000CF92DF92EF92FF920F931F93CF93DF93E7
:102DE0008C01C62FD0E0CE018F579E4F7C01FC0195
:102DF00090819F3F09F447C0D62EF894E92FE295C1
:102E0000EF70F0E081A19F7021E030E001C0220F5F
:102E10009A95EAF7822B81A382A12095282322A3E9
:102E200078940E94A616EDE7F1E041E851E031E028
:102E3000C12C21912F3F89F0A22FA295AF70B0E055
:102E400090968C9190E02F7002C0959587952A9569
:102E5000E2F780FD02C0832F01C080E0C82A330F53
:102E60004E175F0731F7F70180818F3F11F00E9405
:102E7000B11661E0C11001C060E08D2D0E94A8165E
:102E8000C00FD11FC882DF91CF911F910F91FF908A
:102E9000EF90DF90CF9008950E94C81686E0E7EA91
:102EA000F2E0DF01982F1D929A95E9F7E1EAF2E04E
:102EB000DF011D928A95E9F786E00E94A9170C941C
:102EC0002407FF920F931F93CF93DF9300D000D07E
:102ED00000D0CDB7DEB78E010F5F1F4F86E0F8013F
:102EE00011928A95E9F7F12C6F2DC8010E94E8161E
:102EF000F394F6E0FF12F8CF46E050E0B80181EA23
:102F000092E00E94AC2DFF24F394009709F4F12C79
:102F1000892B41F086E0F801A1EAB2E001900D9220
:102F20008A95E1F72F2D46E067EA72E081EA92E0A8
:102F30000E94AA170E9426078F2D26960FB6F89496
:102F4000DEBF0FBECDBFDF91CF911F910F91FF90DC
:102F500008950895FF920F931F93CF93DF938C01F1
:102F6000F62ED72FC42F222349F081E080936C02E4
:102F70000E94812590936B0280936A0280916C027B
:102F80008823C1F080916A0290916B020E9499257A
:102F9000059780F0EF2DFD2FD8014C2F50E0CD018B
:102FA000801B910B841795071CF48D918193F7CFAB
:102FB00010926C02DF91CF911F910F91FF900895B5
:102FC0000E9424280E9475130C9430280E943428F3
:102FD0000E9405140C9452280E941F250E940B2861
:102FE0000E9463130E94E0170E94E6170E946B1371
:102FF000FBCF8091730280FF06C06091090170E0F1
:10300000660F771F2CC081FF08C06091090170E036
:10301000660F771F660F771F22C082FF09C060917D
:10302000090170E043E0660F771F4A95E1F717C08A
:10303000609172026623D1F020910801621778F73F
:103040008091090190E070E033E0880F991F3A9574
:10305000E1F70E94262D622F70E00E94702D6038EB
:10306000710540F46115710519F406C068E070E05F
:10307000862F08958FE7089581E008958091730267
:1030800080FF08C06091050170E0759567957595A2
:10309000679523C081FF06C06091050170E07595BA
:1030A00067951BC082FF04C06091050170E012C0EB
:1030B000609171026623A9F0209104016217A0F7C4
:1030C0008091050170E090E00E94262D622F70E053
:1030D0000E94702D6038710540F46115710519F476
:1030E00006C061E070E0862F08958FE7089581E0C3
:1030F00008958D3E21F40E94F917819504C08E3EFB
:1031000029F40E94F9178093770208958F3E21F4E5
:103110000E94F917819504C0803F29F40E94F91795
:10312000809376020895893F19F40E943E1805C0E5
:103130008A3F31F40E943E18819580937802089569
:103140008B3F21F40E943E18819504C08C3F29F4E6
:103150000E943E188093790208959FE0980F98305E
:1031600078F421E030E0A90102C0440F551F9A9580
:10317000E2F7CA0190917502892B80937502089538
:103180008D3F21F48091730281600BC08E3F21F44A
:1031900080917302826005C08F3F29F48091730291
:1031A00084608093730208958D3E39F49091770284
:1031B00097FF35C01092770259C08E3E29F4909146
:1031C00077021916BCF32BC0909176028F3E29F43A
:1031D00097FF25C01092760249C0803F19F4191656
:1031E000CCF31DC090917802893F29F41916BCF4E4
:1031F000109278023BC08A3F19F497FF10C0F8CFB5
:103200008B3F39F49091790297FF09C010927902AF
:103210002DC08C3F21F4909179021916BCF39FE0E8
:10322000980F983080F421E030E0A90102C0440FEB
:10323000551F9A95E2F7CA018095909175028923EE
:103240008093750213C08D3F21F4809173028E7FAD
:103250000BC08E3F21F4809173028D7F05C08F3F9C
:1032600029F4809173028B7F8093730280917602A0
:10327000811106C080917702811102C01092720202
:1032800080917802811106C080917902811102C07B
:103290001092710208958091690283FF7EC08DEFC4
:1032A00091E00E941F06809175021F928F9388EF14
:1032B00091E09F938F930E94B80686EF91E00E9461
:1032C0001F0680917602282F082E000C330B3F93A7
:1032D0008F9383EF91E09F938F930E94B80681EFC5
:1032E00091E00E941F0680917702282F082E000C83
:1032F000330B3F938F938EEE91E09F938F930E94B9
:10330000B8068CEE91E00E941F0680917802282F6B
:10331000082E000C330B3F938F9389EE91E09F931F
:103320008F930E94B80687EE91E00E941F0680915D
:103330007902282F082E000C330B3F938F9384EED5
:1033400091E09F938F930E94B80681EE91E00E94D6
:103350001F06809172021F928F938EED91E09F93D2
:103360008F930E94B8068CED91E00E941F06809119
:1033700073021F928F9389ED91E09F938F930E9428
:10338000B80686ED91E00E941F068DB79EB74C9659
:103390000FB6F8949EBF0FBE8DBF0E94812520916D
:1033A0007602211104C020917702222321F090930C
:1033B000700280936F0220917802211104C0209145
:1033C0007902222321F090936E0280936D0284E7AC
:1033D00092E00C945F24EF92FF920F931F93CF9390
:1033E000DF9300D000D000D0CDB7DEB786E0E4E7B1
:1033F000F2E0DE01119601900D928A95E1F7E090DE
:103400007602F09077020091780210917902109282
:103410007602109277021092780210927902E110EF
:1034200003C0FF2009F464C080916F029091700284
:103430000E949925FC0120917202222339F080918B
:103440000A0190E08E179F0760F052C080910B0137
:1034500090E06AE070E00E94262D8E179F0718F01A
:1034600047C02F3F19F02F5F20937202EE2061F0CA
:103470000E94F917682F1E1414F08FEF01C081E02D
:103480000E941D2D80937602FF2061F00E94F917A3
:10349000682F1F1414F08FEF01C081E00E941D2DD2
:1034A0008093770280917602882311F12091770230
:1034B0002223F1F0082E000C990B65EB70E00E94BE
:1034C000262D992319F09093760203C081E0809312
:1034D0007602822F220F990B65EB70E00E94262D59
:1034E000992319F09093770203C081E080937702CB
:1034F000011103C0112309F464C080916D02909101
:103500006E020E949925FC0120917102222339F05C
:103510008091060190E08E179F0760F052C0809165
:10352000070190E06AE070E00E94262D8E179F0749
:1035300018F047C02F3F19F02F5F2093710200232E
:1035400061F00E943E18682F101614F08FEF01C032
:1035500081E00E941D2D80937802112361F00E946A
:103560003E18682F111614F08FEF01C081E00E9401
:103570001D2D8093790280917802882311F120918A
:1035800079022223F1F0082E000C990B65EB70E014
:103590000E94262D992319F09093780203C081E0B0
:1035A00080937802822F220F990B65EB70E00E94C6
:1035B000262D992319F09093790203C081E080931E
:1035C00079028091760281110BC08091770281117E
:1035D00007C080917802811103C080917902811126
:1035E0000E944B19EB82FC820D831E8386E0FE0154
:1035F0003196A4E7B2E001900D928A95E1F7269604
:103600000FB6F894DEBF0FBECDBFDF91CF911F91F3
:103610000F91FF90EF900895E4E7F2E086E0DF017C
:103620001D928A95E9F7109272021092710210921F
:103630007302089586E090E00C94B92D682F86E01F
:1036400090E00C94C72D8091AD02847089618093C5
:10365000AD020C941E1B8091AD02869586958695D1
:1036600008958091AD0281FD13C082608093AD0208
:103670000E941E1B8091690280FF08C08DE392E0CA
:103680009F938F930E94B8060F900F900C94BB1DD0
:1036900008958091AD0281FF13C08D7F8093AD02AC
:1036A0000E941E1B8091690280FF08C080E292E0A8
:1036B0009F938F930E94B8060F900F900C94C71D94
:1036C0000895CF93C091AD02C695C17080916902F3
:1036D00080FF0CC01F92CF9389E592E09F938F9358
:1036E0000E94B8060F900F900F900F90CC2319F006
:1036F000CF910C94491BCF910C94311B8091AD025A
:1037000086958170089580910C0108950E94901211
:10371000811104C00E9438130E94231B0E941A1BAF
:103720008093AD02282F26952695269530E02430EB
:10373000310524F0877088618093AD028091AD02DD
:1037400080FF04C086958695869501C080E00C9424
:10375000841D2091AD02822F869586958695482FEF
:1037600050E04330510554F48F5F982F990F990F13
:10377000990F822F8770892B8093AD028091AD02C3
:1037800081608093AD020E941E1B8091690280FFC0
:1037900011C08091AD028695869586951F928F9374
:1037A00080EE92E09F938F930E94B8060F900F9047
:1037B0000F900F908091AD028695869586950C941A
:1037C000841D8091AD02982F969596959695A1F0BF
:1037D000915E990F990F990F8770892B8093AD0295
:1037E000887F91E009F490E08091AD0290FB80F930
:1037F0008093AD020E941E1B8091690280FF11C060
:103800008091AD028695869586951F928F9388EC60
:1038100092E09F938F930E94B8060F900F900F90A5
:103820000F908091AD028695869586950C94841DA7
:103830008091AD0280FD1FC081608093AD02813018
:1038400019F489E08093AD028091AD020E941E1BA5
:103850008091690280FF08C080EA92E09F938F9375
:103860000E94B8060F900F908091AD0286958695C4
:1038700086950C94841D08958091AD0280FF14C03C
:103880008E7F8093AD020E941E1B8091690280FF93
:1038900008C08DE892E09F938F930E94B8060F9026
:1038A0000F9080E00C94841D0895CF93C091AD02D9
:1038B000C1708091690280FF0CC01F92CF9382EB90
:1038C00092E09F938F930E94B8060F900F900F90F5
:1038D0000F90CC2319F0CF910C943C1CCF910C94F9
:1038E000181C9091AD02892F8695869586958F5FDD
:1038F0008F719770843038F4880F880F880F892B68
:103900008093AD0202C09093AD028091AD02887F9A
:1039100091E009F490E08091AD0290FB80F98093F2
:10392000AD020E941E1B8091690280FF11C0809130
:10393000AD028695869586951F928F9389E792E0D2
:103940009F938F930E94B8060F900F900F900F9047
:103950008091AD028695869586950C94841D843061
:1039600008F083E09091AD029770282F220F220F6C
:10397000220F922B9093AD02987F21E009F420E072
:103980009091AD0220FB90F99093AD020C94841DB0
:103990000E94AF1C8091AD020C941E1BFC01DB0148
:1039A00012968C918823F9F0EC5BFC45E730F10529
:1039B000D8F4EA5BFF4F0C94A62D83E001C080E0B1
:1039C0000E94C81C80E008950E94E11BFBCF0E946A
:1039D000A91BF8CF0E94551CF5CF0E94711CF2CF95
:1039E0000E94611BEFCF81E00895279A2F980895D8
:1039F0002F9808958F929F92AF92BF92CF92DF92AD
:103A0000EF92FF920F931F93CF93DF938C018091DE
:103A10008600909187006CE070E00E945C2D60173A
:103A2000710730F0C80169E070E00E945C2D5EC053
:103A30008091860090918700E0908600F09087004A
:103A4000E0918600F0918700C6E0D0E0BE010E94C0
:103A50005C2D20E030E0060F171F211D311D4801AD
:103A6000590185E0880C991CAA1CBB1C8A95D1F7CA
:103A7000C701BE010E945C2D6F01E12CF12CA70152
:103A80009601260F371F411D511DC501B4010E942B
:103A9000842D69017A01C0918600D0918700CA0106
:103AA000B9010E94372D9E0140E050E00E94372D61
:103AB000A70196010E94372DDC01CB012FE0B695BE
:103AC000A795979587952A95D1F700918600109133
:103AD000870020E030E0081719072A073B0728F481
:103AE0006091860070918700CB01BC01CB01DF9112
:103AF000CF911F910F91FF90EF90DF90CF90BF90EB
:103B0000AF909F908F900895CF93C82F843050F43A
:103B1000811109C080918000877F809380000E947E
:103B2000F81C06C0C3E0809180008860809380000C
:103B3000609186007091870080E090E02C2F30E04B
:103B400040E050E00E94372D23E030E040E050E0BC
:103B50000E94842DB42FA32F922F8827892F9A2F6C
:103B6000AB2FBB270E94FA1C90938D0080938C0092
:103B7000CF910895089510927B0210927A021092CC
:103B80007C02EFE6F0E08081816080830895EFE6BB
:103B9000F0E080818E7F80830E942B1B0C94841D1B
:103BA0001F920F920FB60F9211240F931F932F9312
:103BB0003F934F935F936F937F938F939F93AF93B5
:103BC000BF93CF93DF93EF93FF9380910D0191E02B
:103BD000980F823019F090930D015BC081E08093C3
:103BE0000D010E94831B182FC0917A02D0917B0295
:103BF00021960E94831B90E068E770E00E94262DCA
:103C0000BC01CE010E945C2D9C0190937B028093AD
:103C10007A02812F90E068E770E00E94262DBC01B7
:103C2000660F672F661F770B7195C9010E945C2D87
:103C30006F7780917C02823019F4603451F404C0B3
:103C4000813039F46F3729F480916F008E7F809333
:103C50006F00E62FF0E0E850FD4FC4910091860020
:103C6000109187000E942B1B282F8C2F90E0B80109
:103C70000E94262D6DEF72E00E945C2DCB01622F19
:103C800070E00E94262D0E94FA1C90938D00809374
:103C90008C00FF91EF91DF91CF91BF91AF919F91F8
:103CA0008F917F916F915F914F913F912F911F91D4
:103CB0000F910F900FBE0F901F9018950E94F51C4A
:103CC0008AE08093800089E1809381008FEF9FEFED
:103CD00090938700809386000E94861B0E947E1B23
:103CE00081110C94BB1D0895CF93DF93EC01FB0170
:103CF0008281882309F43CC1C430FDE5DF0760F40C
:103D0000CB3F9CE5D90788F49E0122503C452431E5
:103D1000310508F02EC109C0C236EDE5DE0729F0F5
:103D2000C63AFDE5DF0709F024C10E94A312909373
:103D3000A00280939F02C1318CE5D80709F4C6C068
:103D400008F042C0C930ECE5DE0709F49BC000F57D
:103D5000C5308CE5D80709F485C078F4C330ECE5AC
:103D6000DE0709F478C008F07AC0C230DC4509F0FB
:103D7000F5C080919F028160EFC0C7309CE5D907F4
:103D800009F478C008F07AC080919F028061E4C095
:103D9000CD30FCE5DF0709F487C058F4CB309CE553
:103DA000D90709F479C008F07BC080919F02886030
:103DB0006FC0CF30FCE5DF0709F480C008F082C097
:103DC00080919F02877FC8C0CE3F9CE5D90709F448
:103DD00071C000F5C531FCE5DF0709F485C068F462
:103DE000C3319CE5D90709F475C008F095C00E945D
:103DF000410C80919F028F77AFC0CC3FFCE5DF077D
:103E0000A9F108F054C0CB3FDC4509F0A7C0809170
:103E1000A00240C0C230EDE5DE0709F489C058F4C5
:103E2000C1158DE5D80709F45AC008F069C0809122
:103E3000A00282602FC0C236EDE5DE0709F47CC027
:103E4000C63AFDE5DF0709F481C0C330DD4509F05E
:103E500085C080E06EC080919F0282607DC08091AD
:103E60009F0216C080919F02886076C08091A00258
:103E700082604FC080919F0280626EC080919F02DD
:103E800080646AC00E94410C80919F02806864C077
:103E9000846062C081603DC080919F028E7F5CC063
:103EA00080919F028D7F58C080919F0216C08091A3
:103EB000A00218C08091A0028D7F2BC080919F022C
:103EC0008F7E4AC080919F028F7D46C080919F0265
:103ED0008F7B42C080919F02877F8B7F3DC0809106
:103EE000A0028D7F8E7F15C080919F0282FB2227CA
:103EF00020F991E0922790FB82F990FB83F92CC086
:103F00008091A002982F909591708E7F892B90FBC5
:103F100081F98093A00222C00E94410C80919F02EF
:103F200087FB222720F991E0922790FB87F914C0A4
:103F300081E00E943A1312C080919F0284FB2227E5
:103F400020F991E0922790FB84F906C080919F02AE
:103F5000982F909590FB80F980939F0280919F020B
:103F60009091A0020E94B4120E94410C80E001C016
:103F700081E0DF91CF910895809104011F928F938A
:103F8000809105011F928F93809108011F928F935A
:103F9000809109011F928F9380910A011F928F9344
:103FA00080910B011F928F9388E793E09F938F93EB
:103FB0000E94B8068DB79EB70E960FB6F8949EBFB6
:103FC0000FBE8DBF0895883220F58E3108F068C08D
:103FD0008B3091F1C0F4873009F0BEC081E080934E
:103FE0000B0184E180930A018AE0809309018EE14C
:103FF0008093080188E08093050188E280930401A2
:104000008AED94E0C6C0833109F443C0843169F17C
:10401000A3C08F3409F49EC028F4893231F188336B
:1040200059F09AC0813531F008F4D4C0823509F4D2
:10403000A7C092C08FEFA5C08CEF94E00E941F062E
:104040000E94BC1F1F9281E08F931F9288E08F9384
:1040500085EF93E09F938F930E94B8060F900F9087
:104060000F900F900F900F9096C089EF94E00E94F0
:104070001F0680918102882309F4AAC01092810250
:104080001092800210927F0210927E0210927D02A6
:10409000B1C08BEE94E00E941F060E94BC1F7BC043
:1040A0008D5180938102833031F170F48130D1F0F1
:1040B000823009F03FC08AE091E0909380028093C3
:1040C0007F0284E991E01FC0853059F108F1863004
:1040D00089F584E091E09093800280937F028FECD9
:1040E00091E011C08BE091E09093800280937F0279
:1040F0008BE891E008C089E091E090938002809382
:104100007F0280EA91E090937E0280937D0218C046
:1041100088E091E09093800280937F028DEA91E0A5
:10412000F2CF85E091E09093800280937F028CEB48
:1041300091E0E9CF1092810288EE94E00E941F0680
:1041400080918102882309F455C01F928F9384EED9
:1041500094E00DC08AE015C087ED94E01AC097FF87
:1041600047C0108280811F928F9381ED94E09F93CE
:104170008F930E94B8060F900F900F900F900BC076
:1041800081E0E0917F02F0918002309729F58EEC7A
:1041900094E00E941F0620918102222359F1809110
:1041A0007D0290917E02009711F487E891E09F9341
:1041B0008F931F922F9385EC94E09F938F930E948F
:1041C000B8060F900F900F900F900F900F9016C0A1
:1041D00080E0089586EFD5CF2081082E000C990B42
:1041E000820F911D8F3F910509F00CF4B8CF8FEF2E
:1041F0008083B8CF81EC94E00E941F0681E008958F
:10420000CF93C82F1F928F9382E195E09F938F9356
:104210000E94B80681E090E0A0E0B0E0BC01CD01D2
:1042200004C0660F771F881F991FCA95D2F70E9496
:10423000990C0F900F900F900F90CF910C94410C10
:10424000EF92FF920F931F93CF93DF938B3109F47B
:1042500009C108F0AAC08B3009F4CDC008F094C0A1
:10426000863009F4CBC020F4853009F4D9C06AC186
:10427000873009F4DCC0883009F064C10E949F12C5
:104280001F928F9383E699E09F938F930E94B806C5
:104290000E949B1283FB992790F91F929F9382FBA8
:1042A000992790F91F929F9381FB992790F91F926C
:1042B0009F93982F91701F929F931F928F938AE1E3
:1042C00099E09F938F930E94B8060E94A31287FBE8
:1042D000222720F91F922F9386FB222720F91F9275
:1042E0002F9385FB222720F91F922F9384FB2227EF
:1042F00020F91F922F9383FB222720F91F922F93DF
:1043000082FB222720F91F922F9391FB222720F96D
:104310001F922F93292F21701F922F9381FB222709
:1043200020F91F922F93282F21701F922F939F9374
:104330008F9385E398E09F938F930E94B8068DB783
:104340009EB788960FB6F8949EBF0FBE8DBF0E9491
:104350001A1B982F9695969596951F929F93982F36
:1043600091701F929F931F928F9382E098E09F938A
:104370008F930E94B8068DB79EB708960FB6F89433
:104380009EBF0FBE8DBF35C0803109F495C020F4AB
:104390008E3009F47BC0D6C0863109F4A8C08931BB
:1043A00009F0D0C082E895E084C08A32E1F060F480
:1043B000873209F4C3C028F48E3108F4C3C08D518C
:1043C000BEC0893269F1BEC0833448F48A3308F034
:1043D000B3C0853309F4B2C0883369F0B3C0833405
:1043E00009F4ACC0AFC08EE09AE00E941F060E94A4
:1043F0003813C1E0ACC08FE596E05BC080916902E4
:10440000817F8E7F8093690288E396E00E941F0679
:104410008AE09AE00E941F0681E080938202E9CF41
:104420008EEE99E00E941F060E942907E2CF80913C
:104430006902C82FC095C170C0FB80F980936902E2
:10444000CC2329F082EE99E00E941F0680C085ED02
:1044500099E00E941F0680916902897F877F80937F
:104460006902C7CF9091690291FBCC27C0F981E026
:10447000C827892FC0FB81F980936902CC2319F0EA
:1044800088EC99E029C08AEB99E013C09091690209
:1044900092FBCC27C0F981E0C827892FC0FB82F9A5
:1044A00080936902CC2319F08BEA99E015C08BE95F
:1044B00099E00E941F069DCF9091690293FBCC2743
:1044C000C0F981E0C827892FC0FB83F98093690276
:1044D000CC2351F08FE899E00E941F068091690279
:1044E00081608093690233C082E899E0E2CF0E9444
:1044F0008D25162F072FF82EE92ED0919E02C09100
:104500001A010E940A24EF92FF920F931F931F92A9
:10451000DF931F92CF931F928F9387E195E09F9334
:104520008F930E94B8068DB79EB70C960FB6F8947D
:104530009EBF0FBE8DBF5DCF895301C080E00E943A
:10454000002157CF80E899E00E941F06C0E08C2F21
:10455000DF91CF911F910F91FF90EF90089580E030
:1045600008950C94AF22CF93C82F8091820281309E
:1045700071F040F0823009F045C08C2F0E94E31F9B
:1045800081E046C00E9493118232F1F504C00E947E
:104590009311823261F48C2F0E94B122811104C0E8
:1045A0008C2F0E9420212CC081E090E029C08C2F0C
:1045B0000E94AF22811123C0C431C9F058F4CB301E
:1045C00069F0C031B9F482E08093820288E30E94EE
:1045D000E31F15C0C93259F0C83361F488E396E08F
:1045E0000E941F068EE095E00E941F0608C01092F0
:1045F00082020CC08CE095E00E941F0607C081E09B
:10460000817006C01092820280E002C080E0F8CF84
:10461000CF910895CF93DF9386319C4541F5EB010F
:104620000E949311982F8A812091020130910301F9
:10463000882379F09A7A81E009F480E080938302FC
:10464000911102C069E201C065E3C9010E94DB2447
:104650000AC080918302811102C069E201C065E352
:10466000C9010E94DD240E94D51180E001C081E0D3
:10467000DF91CF9108950F931F93CF93DF93C42FB2
:10468000D22FFC0182818823C9F0409386020E94C8
:104690008125909385028093840280E28C0F88307C
:1046A00008F057C0C77081E001C0880FCA95EAF7CB
:1046B000DF91CF911F910F910C949E0980918602FA
:1046C000481330C080918402909185020E94992500
:1046D000883C910538F510E21D0FCD17B9F080E246
:1046E0008C0F883040F4C77081E001C0880FCA95F4
:1046F000EAF70E94A509183028F581E09D2F9770F0
:1047000001C0880F9A95EAF70E949E09802F0E94A7
:1047100095091830F0F4D77081E001C0880FDA9560
:10472000EAF70AC080E28C0F883098F4C77081E005
:1047300001C0880FCA95EAF7DF91CF911F910F91C1
:104740000C94A509802FDF91CF911F910F910C94AC
:104750009509DF91CF911F910F9108950F939C01BF
:10476000CB01243F4CE5340731F188F4293DFCE5C9
:104770003F07D9F02A3D4CE5340779F1283D3C4507
:10478000A9F506E221EE41EE68ED7CE52BC0263F5F
:10479000FCE53F07E1F0A8F0273F3C4539F507E28B
:1047A00025EE46EE67EF7CE51DC007E225EE45EEFF
:1047B00069ED7CE517C006E221EE40EE64EF7CE592
:1047C00011C007E225EE44EE65EF7CE50BC006E282
:1047D00021EE42EE66EF7CE505C008E221E045EE01
:1047E0006AED7CE50E943B2380E008C0FC018281E9
:1047F000882319F01092860201C081E00F9108957C
:104800009093F5018093F401089590938C02809326
:104810008B020895E0918B02F0918C02309721F089
:104820000190F081E02D099480E00895EF92FF92CD
:104830000F931F93CF93DF93E0918B02F0918C0243
:104840003097B1F18C010280F381E02D09958091C0
:10485000690282FF2DC080FF04C087E29AE00E94B7
:104860001F06E80118E081E2E82E8AE0F82E809128
:10487000690280FF0BC088811F928F93FF92EF9295
:104880000E94B8060F900F900F900F901150219634
:104890001111EDCF8091690280FF0AC08FE19AE08B
:1048A000DF91CF911F910F91FF90EF900C941F0615
:1048B000DF91CF911F910F91FF90EF900895E091BC
:1048C0008B02F0918C02309739F022E0DC012C93BE
:1048D0000480F581E02D099408952091890230919A
:1048E0008A022817390771F090938A02809389020F
:1048F000E0918B02F0918C02309721F00680F781D5
:10490000E02D09940895209187023091880228179C
:10491000390771F09093880280938702E0918B02AF
:10492000F0918C02309721F00084F185E02D0994FC
:104930000895FC01329697E080E0915029F0219192
:104940002223D9F38F5FF9CF0895662349F0FC0144
:10495000329608962191621729F0E817F907D1F7E6
:1049600080E0089581E008959C01FC0132969FEF5C
:1049700080E04191461789F09F3F19F4411101C031
:10498000982F8F5F8630A9F79F3F39F0F901E90F23
:10499000F11D97FDFA956283089508959C012A5FA1
:1049A0003F4FFC014281461301C0128201968217DB
:1049B0009307B9F708950C94B4240C94CE2402966E
:1049C00026E0FC0111922A95E9F7089508950C94C8
:1049D000E62483E080938D020C94E724811102C0C9
:1049E00081E001C082E080938D020C94E7240C9456
:1049F000EE2481E080938D020C94E7240C94F9243A
:104A000008950C9400250C9401250C9400250C9419
:104A100000250C940025CF930E9407250E94611762
:104A20000E940525C0E08C2F0E945616811104C0FB
:104A3000CF5FC630C1F701C081E0CF9108950895DE
:104A40001F920F920FB60F9211248F939F93AF93E3
:104A5000BF9380918E02811113C08091AE0290911C
:104A6000AF02A091B002B091B1024196A11DB11D5B
:104A70008093AE029093AF02A093B002B093B102C4
:104A8000BF91AF919F918F910F900FBE0F901F908C
:104A900018958091B602843031F10E94B0071092CF
:104AA0008E0220E488E190E00FB6F894A8958093F8
:104AB00060000FBE2093600083B7817F846083BF56
:104AC00083B7816083BF7894889583B78E7F83BFD7
:104AD0000FB6F894A895809160008861809360007B
:104AE000109260000FBE08950E94410C0C94B7070D
:104AF00082E084BD93E095BD9AEF97BD80936E00F0
:104B000008952FB7F8948091AE029091AF02A091D2
:104B1000B002B091B1022FBF08952FB7F894609101
:104B2000AE027091AF028091B0029091B1022FBF9E
:104B300008959C014FB7F8948091AE029091AF0216
:104B4000A091B002B091B1024FBF821B930B0895A8
:104B500078941F920F920FB60F9211248F939F9308
:104B6000AF93BF938091AE029091AF02A091B0023B
:104B7000B091B1020196A11DB11D8093AE02909338
:104B8000AF02A093B002B093B102BF91AF919F91D9
:104B90008F910F900FBE0F901F90189581E080931A
:104BA000E00080E28093D8001092C9008FE19EE47B
:104BB0000197F1F700C0000087E090EBDC018093E3
:104BC000BF029093C002A093C102B093C2029CE0C6
:104BD00088E10FB6F894A895809360000FBE90937B
:104BE0006000FFCF80919D020895089522E02093F8
:104BF000E9002FEF3091E800215035FD06C035ED7A
:104C00003A95F1F700002111F5CF2091E80025FF3A
:104C10000BC040E050E066E070E00E94C128809147
:104C2000E8008E778093E8000895CF93DF9321E02A
:104C30002093E9002FEF3091E800215035FD06C0A8
:104C400035ED3A95F1F700002111F5CF2091E800FC
:104C500025FF14C0EC0140E050E068E070E00E94E5
:104C6000C1288091E8008E778093E80088E0FE01FB
:104C7000A5E9B2E001900D928A95E1F7DF91CF911D
:104C800008958093910270939302609392028091B1
:104C9000B602843001F582E08093E9008FEF9091B5
:104CA000E800815095FD06C095ED9A95F1F700005A
:104CB0008111F5CF8091E80085FF0DC040E050E004
:104CC00063E070E081E992E00E94C1288091E800F1
:104CD0008E778093E8000895BC0184E00C9441260F
:104CE000BC0183E00C94412685E49AE00E941F06F3
:104CF0000C94FE2481E49AE00E941F066091B202A7
:104D000081E0611101C080E00C94E9248DE39AE018
:104D10000E941F069091B60281E0943009F080E075
:104D20006091B2020C94EE24209190022F5F822FAA
:104D300062E30E94502D992319F020939002089568
:104D40001092900280919402882371F18091B602B2
:104D5000843041F58091E9008F702091EC00922F12
:104D6000917020FD90E8892B93E09093E900909159
:104D7000EB0090FF14C09091EE0097FF10C090914F
:104D8000E80095FF03C01092F100F9CF9091E80080
:104D900090FF05C09091E8009E779093E8008F7097
:104DA0008093E90010929402089542E061EC81E062
:104DB0000E94C52942E261EC82E00E94C52942E2DC
:104DC00061EC83E00E94C5299091B60281E09430A5
:104DD00009F080E06091B2020C94F7248091B8024F
:104DE000833009F45DC030F4813071F0823009F411
:104DF00096C008958A3009F482C08B3009F468C0E7
:104E0000893009F0A4C020C08091B702813A09F02E
:104E10009EC08091E800877F8093E8008091BB026C
:104E20009091BC02892B21F468E085E992E003C0EF
:104E300060E080E090E070E00E940C298091E80042
:104E40008B778093E80008958091B702813209F052
:104E50007EC08091BB029091BC02029708F077C09F
:104E60008091E800877F8093E8008091E80082FDD0
:104E700005C08091B6028111F8CF69C08091F2001F
:104E8000823031F48091F100813011F0863021F4CC
:104E90008091F10080939D028091E8008B7753C050
:104EA0008091B702813A09F052C08091BB02909183
:104EB000BC02892B09F04BC08091E800877F80936A
:104EC000E8008091E80080FFFCCF80911A0136C095
:104ED0008091B7028132D9F58091BB029091BC02DA
:104EE000892BA9F58091E800877F8093E8000E94D4
:104EF000FA298091B90280931A010C94410C809197
:104F0000B702813221F58091E800877F8093E80025
:104F10000E94FA298091BA0280939E02089580919E
:104F2000B702813AA1F48091E800877F8093E8007E
:104F30008091E80080FFFCCF80919E028093F10079
:104F40008091E8008E778093E8000C94FA29089508
:104F50009FB7F894109294029FBF9091B60294303C
:104F600009F057C09091E9009F703091EC00232F19
:104F7000217030FD20E8922B23E02093E90020915E
:104F8000EB0020FF43C02091EE0027FF3FC020919F
:104F90008F02222321F02091E80025FF37C01092D4
:104FA0008F0226E03091E80035FD15C03091B60241
:104FB000343061F53091EB0035FD28C0215021F4EB
:104FC00081E080938F0222C0EFE9FFE03197F1F793
:104FD00000C00000E7CF8093F1008091E80085FDDC
:104FE0000AC08091E80080FFFCCF8091E8008E77B6
:104FF0008093E80006C08FB7F89421E020939402D4
:105000008FBF9F709093E90080E008959F70909308
:10501000E9008FEF089584B7877F84BF0FB6F894B7
:10502000A895809160008861809360001092600074
:105030000FBE90E080E80FB6F894809361009093E3
:1050400061000FBE0C94F9240E944C2A0E949F2AF2
:10505000E2EEF0E080818460808378940C94022DED
:105060008EE091E00C9405248091B6028530C9F45D
:1050700089E39AE00E941F068091B602853079F498
:105080000E9449258091B4028823B1F30E940B2528
:10509000882391F30E94AB280E94410CEDCF0C9421
:1050A0007425089508950C945528292F332723300B
:1050B0003105C9F060F42130310581F0223031052D
:1050C00009F041C08BE590E027E63AE040C021328C
:1050D0003105E1F02232310531F135C082E190E055
:1050E00022EC3AE034C099278130910549F028F04C
:1050F000029749F5E9E4FAE005C0E3E6FAE002C008
:10510000E3E5FAE0849190E09F0121C063307105EE
:10511000D0F4660F771FFB01E351FE4F20813181F0
:1051200089E090E014C06330710568F4FB01EE0F74
:10513000FF1FE951FE4F20813181FB01EC51FE4FF1
:10514000808190E004C080E090E020E030E0FA014F
:1051500031832083089584E089BD86E089BD09B448
:1051600000FEFDCF8091D8008F7D8093D800809184
:10517000E00082608093E0008091E00081FDFCCF40
:105180000895CF92DF92EF92FF920F931F93CF93E8
:10519000DF93EC018B017A010E94192A811133C03F
:1051A000E114F10439F0F70180819181081B190B9A
:1051B000C80FD91FC12CD12C0115110519F18091EF
:1051C000E80085FD16C08091E8008E778093E800A6
:1051D000E114F10449F0F70180819181C80ED91ED4
:1051E000D182C08285E00FC00E94192A882321F352
:1051F0000AC089918093F10001501109FFEFCF1A85
:10520000DF0ADACF80E0DF91CF911F910F91FF90FD
:10521000EF90DF90CF9008952091BD023091BE02B3
:105220002617370748F06115710539F42091E80019
:105230002E772093E80001C0B901FC0120E0611540
:10524000710561F18091B6028823D9F18530D9F1D9
:105250008091E80083FD39C08091E80082FD2BC079
:105260008091E80080FFEBCF8091F20090E0611523
:10527000710551F08830910538F421912093F100A7
:10528000615071090196F3CF21E0089709F020E001
:105290008091E8008E778093E800D1CF2111D2CFA2
:1052A0000AC08091B602882361F0853061F0809158
:1052B000E80083FD0AC08091E80082FFF2CF80E021
:1052C000089582E0089583E0089581E00895209193
:1052D000BD023091BE022617370748F061157105EF
:1052E00039F42091E8002E772093E80001C0B9013D
:1052F000FC0120E06115710579F18091B6028823E7
:1053000009F43DC0853009F43CC08091E80083FD7C
:105310003AC08091E80082FD2CC08091E80080FFB7
:10532000E9CF8091F20090E06115710559F0883065
:10533000910540F424912093F10031966150710958
:105340000196F2CF21E0089709F020E08091E80073
:105350008E778093E800CECF2111CFCF0AC0809105
:10536000B602882361F0853061F08091E80083FD0A
:105370000AC08091E80082FFF2CF80E0089582E0C9
:10538000089583E0089581E00895982F953068F599
:105390009093E900981739F07091EC002091ED009E
:1053A0005091F00003C0242F762F50E021FD02C061
:1053B0009F5FECCF3091EB003E7F3093EB0030915C
:1053C000ED003D7F3093ED003091EB003160309384
:1053D000EB007093EC002093ED005093F0002091CF
:1053E000EE0027FDE5CF80E008958F708093E900FF
:1053F00081E008958091B70287FF11C08091E80095
:1054000082FD05C08091B6028111F8CF11C0809154
:10541000E8008B770BC08091B602882349F0809119
:10542000E80080FFF8CF8091E8008E778093E80055
:1054300008952091E4003091E50095E64091EC005C
:10544000842F817040FF23C08091E80080FD1DC043
:105450008091B602882399F0853099F08091EB0015
:1054600085FD11C04091E4005091E50024173507F7
:1054700029F3915011F09A01E1CF84E0089582E080
:10548000089583E0089581E0089580E008954091B3
:10549000E80042FFDDCF08950E94A92A0E94AC2AAD
:1054A000E0EEF0E0808181608083E8EDF0E08081D3
:1054B0008F77808319BCE3E6F0E080818160808390
:1054C0001092B50208950E94A92A0E94AC2A8091E8
:1054D000D8008F778093D8008091D800806880931F
:1054E000D8008091D8008F7D8093D80084E089BD5A
:1054F00086E089BD09B400FEFDCF1092B60210927D
:10550000B2021092B4021092B30242E060E080E076
:105510000E94C5298091E1008E7F8093E1008091F7
:10552000E20081608093E2008091E20088608093D5
:10553000E2008091E0008E7F8093E0000895E3E632
:10554000F0E080818E7F808381E08093B5020C94AF
:10555000632A1092E20008951092E10008951F92CC
:105560000F920FB60F9211242F933F934F935F9397
:105570006F937F938F939F93AF93BF93EF93FF931B
:105580008091E10082FF0BC08091E20082FF07C0A2
:105590008091E1008B7F8093E1000E9494268091AE
:1055A000E10080FF19C08091E20080FF15C080916A
:1055B000E2008E7F8093E2008091E2008061809320
:1055C000E2008091D80080628093D80019BC85E009
:1055D0008093B6020E947A268091E10084FF30C059
:1055E0008091E20084FF2CC084E089BD86E089BD03
:1055F00009B400FEFDCF8091D8008F7D8093D80044
:105600008091E1008F7E8093E1008091E2008F7EA7
:105610008093E2008091E20081608093E2008091BB
:10562000B202882311F084E007C08091E30087FD77
:1056300002C081E001C083E08093B6020E9486260A
:105640008091E10083FF29C08091E20083FF25C0A3
:105650008091E100877F8093E10082E08093B60231
:105660001092B2028091E1008E7F8093E1008091E0
:10567000E2008E7F8093E2008091E200806180935F
:10568000E20042E060E080E00E94C5298091F000E5
:1056900088608093F0000E947426FF91EF91BF9183
:1056A000AF919F918F917F916F915F914F913F91BA
:1056B0002F910F900FBE0F901F9018951F920F9271
:1056C0000FB60F9211242F933F934F935F936F93D5
:1056D0007F938F939F93AF93BF93CF93DF93EF937A
:1056E000FF93C091E900CF708091EC00D82FD1706A
:1056F00080FDD0E81092E9008091F000877F8093D0
:10570000F00078940E94A22B1092E9008091F000A2
:1057100088608093F000CD2BCF70C093E900FF919B
:10572000EF91DF91CF91BF91AF919F918F917F9139
:105730006F915F914F913F912F910F900FBE0F90FE
:105740001F9018951F93CF93DF93CDB7DEB7AA971D
:105750000FB6F894DEBF0FBECDBFE7EBF2E080914D
:10576000F100819322E0EF3BF207C9F70E94EE2699
:105770008091E80083FF2EC18091B7029091B8021A
:10578000492F50E04A30510508F024C1FA01E35B8B
:10579000FF4F0C94A62D803821F0823809F01AC1F1
:1057A00008C08091B3029091B402992389F082607D
:1057B0000FC08091BB028F70853008F00BC18093C1
:1057C000E9008091EB0085FB882780F91092E900C1
:1057D0009091E800977F9093E8008093F1001092F9
:1057E000F100D1C0282F2D7F09F0F4C0882319F0D3
:1057F000823061F0EFC08091B902813009F0EAC0D7
:10580000933009F080E08093B4022EC08091B902F9
:1058100081112AC08091BB028F702FEF280F243096
:1058200008F0D8C08093E9002091EB0020FF1CC055
:10583000933021F48091EB00806214C09091EB00D2
:1058400090619093EB0021E030E0A90102C0440F89
:10585000551F8A95E2F74093EA001092EA00809182
:10586000EB0088608093EB001092E9008091E800E3
:10587000877F8093E8000E94FA29ACC08111AAC0FA
:105880001091B9021F778091E3008078812B80937B
:10589000E3008091E800877F8093E8000E94FA2966
:1058A0008091E80080FFFCCF8091E30080688093C6
:1058B000E300111102C082E001C083E08093B602D0
:1058C00089C08058823008F085C08091B9029091DB
:1058D000BA028C3D53E0950779F583E08A838AE22A
:1058E00089834FB7F894DE01139620E03EE051E241
:1058F000E32FF0E050935700E49120FF03C0E295BE
:10590000EF703F5FEF708E2F90E0EA3010F0C79697
:1059100001C0C0968D939D932F5F243149F74FBFEF
:105920008091E800877F8093E8006AE270E0CE0112
:1059300001960E940C2916C06091BB027091BC02B6
:10594000AE014F5F5F4F0E945328BC01892B09F4C1
:1059500041C09091E800977F9093E80089819A81F7
:105960000E9467298091E8008B778093E80032C01D
:10597000803881F58091E800877F8093E8008091EE
:10598000B2028093F1008091E8008E7772CF81118E
:1059900021C08091B9029091BA0299270297D4F45C
:1059A0008091E800877F8093E8008091B90280931E
:1059B000B2020E94FA298091B202811106C0809140
:1059C000E30087FD02C081E001C084E08093B6025D
:1059D0000E94D5268091E80083FF0AC08091E800EC
:1059E000877F8093E8008091EB0080628093EB00DA
:1059F000AA960FB6F894DEBF0FBECDBFDF91CF9150
:105A00001F910895CF938091B6028823A1F0C09191
:105A1000E900CF709091EC00892F817090FD80E8B3
:105A2000C82B1092E9008091E80083FD0E94A22B10
:105A3000CF70C093E900CF910895002480FD060E39
:105A4000660F11F08695D1F7802D08950024552713
:105A500004C0080E591F880F991F009729F07695EA
:105A60006795B8F37105B9F7802D952F0895EE2746
:105A7000FF27AA27BB2708C0A20FB31FE41FF51FEB
:105A8000220F331F441F551F96958795779567956D
:105A900098F37040A9F7009799F7BD01CF010895D9
:105AA000991B79E004C0991F961708F0961B881F70
:105AB0007A95C9F780950895AA1BBB1B51E107C0D1
:105AC000AA1FBB1FA617B70710F0A61BB70B881F8E
:105AD000991F5A95A9F780959095BC01CD0108951D
:105AE00097FB072E16F4009407D077FD09D00E948B
:105AF0005C2D07FC05D03EF4909581959F4F08954D
:105B0000709561957F4F0895A1E21A2EAA1BBB1BC9
:105B1000FD010DC0AA1FBB1FEE1FFF1FA217B30779
:105B2000E407F50720F0A21BB30BE40BF50B661F8F
:105B3000771F881F991F1A9469F760957095809553
:105B400090959B01AC01BD01CF010895EE0FFF1FA1
:105B50000590F491E02D0994FB01DC0104C08D91C6
:105B60000190801921F441505040C8F7881B990BCF
:105B70000895F999FECF92BD81BDF89A992780B515
:105B80000895A8E1B0E042E050E00C94ED2D262FFE
:105B9000F999FECF92BD81BDF89A019700B4021623
:105BA00039F01FBA20BD0FB6F894FA9AF99A0FBED1
:105BB00008950396272F0E94C82D0E94C72D252FD8
:105BC0000E94C82D242F0C94C82D0196272F0E94C7
:105BD000C82D0C94C72DDC01CB01FC01F999FECF37
:105BE00006C0F2BDE1BDF89A319600B40D92415065
:0A5BF0005040B8F70895F894FFCF75
:105BFA00C8005102280850011E0A14010601F225A4
:105C0A001526F62570266C26F52501E200E900EA3C
:105C1A0000B500B600B700CD008301CC008A01921E
:105C2A000194012102230224022502260227022AC4
:105C3A0002B300B4006F007000818283E200E900C1
:105C4A00EA00B500B600B700CD008301CC008A0196
:105C5A00920194012102230224022502260227022C
:105C6A002A02B300B4006F00700081828334659207
:105C7A00916430939495963F3F3F006D6B5F6465E6
:105C8A006C6179006D6B5F696E74657276616C0028
:105C9A006D6B5F6D61785F7370656564006D6B5FD6
:105CAA0074696D655F746F5F6D6178006D6B5F77A6
:105CBA006865656C5F6D61785F7370656564006DBA
:105CCA006B5F776865656C5F74696D655F746F5F3C
:105CDA006D617800407B22710BF60AD40A790A9228
:045CEA000AAB0A00F7
:00000001FF
